:020000040000FA
:0400000080312428FF
:100008007E1480310B1D09280A2822280B11F101C2
:100018000130F00070082000A207221C14281528BF
:100028001C282508031919281A281C28F101F10A87
:10003800710C2200031C8E1003188E147E10090008
:10004800803126288731FD278031CA008731FE2775
:100058008031CB00FA01FB0120308400003085009C
:1000680017308F31CF278031CA30840000308500A7
:100078000A308F31CF2780317E10200081313F290F
:100088002000C300420883313623803120003E0817
:100098003F04031950285128F62886314D2680310F
:1000A80072087304031959285A288C28200042081A
:1000B80085316B258031720873040319642865281B
:1000C800782887316927803187315027803100307F
:1000D80085319425803100308631F8268031013011
:1000E8008731162780313E2987316927803187314A
:1000F8005027803101308531942580310030863198
:10010800F8268031200024088731162780313E29BF
:100118002000420885316B25803172087304031969
:1001280096289728AA288731692780318731502750
:100138008031003085319425803100308631F826B1
:10014800803101308731162780313E2986312926B2
:10015800803177087804031DB228B328C628863171
:10016800B826803187315027803100308531942579
:10017800803100308631F8268031013087311627EA
:1001880080313E2984312A248031863129268031E4
:10019800770878040319D128D228E2288731502714
:1001A8008031003085319425803100308631F82641
:1001B800803101308731162780313E298731692700
:1001C8008031873150278031013085319425803145
:1001D80000308631F8268031200024088731162720
:1001E80080313E29430885314225803172087304E5
:1001F8000319FF28002903298331782380318631A8
:10020800052680317708780403190B290C29202941
:1002180087316927803100308531942580318731D5
:100228003427803176088631F8268031200023086B
:100238008731162780313E298731692780318731F8
:100248005027803100308531942580310030863147
:10025800F82680312000420885316B2580317208EC
:100268007304031D38293A2901303B2900308731AE
:100278001627803108008331F12381312D308731F1
:10028800AC27813128308731AC278131CA3087319A
:10029800AC278131A030F2000F30F300CA3087312B
:1002A80097278131B6308431C0248131C030843100
:1002B800C0248131A2308431EC248131AC308431C6
:1002C800EC2481318731EF2781318731E127813172
:1002D80085311825813173082000C6007208C500D1
:1002E8007A304602123003194502031C7C297D2905
:1002F8008F298731EF2781312000C501C6010130E0
:10030800CA000030CB000130F4000030F500823123
:10031800AB22813195290030F400F5008231AB22FF
:10032800813120004B08F3004A08F2007D30F400C8
:100338000030F5008631D926813173082100A100EB
:100348007208A0008631952681318231F2228131EE
:100358008531BC258131AC302000C4004408B70089
:10036800A230863171268131C0302000C400440893
:10037800B700B6308531E12581318431932481314C
:10038800C0302000C4004408F800B6308731D127B7
:1003980081310130FA000030FB00A2302000C40097
:1003A8004408C200B6308031442081310230FA005E
:1003B8000030FB00AC302000C4004408C200C0304C
:1003C80080314420813187318227813177082000AC
:1003D800C400C40DC40D22000C0820004406FB39DB
:1003E800440622008C00853118258131210021081E
:1003F8007302031D012A20087202031C042A052A1D
:10040800F72901302000CA070030CB3D6929803127
:100418002428F900720873040319132A142A632A7A
:100428007908023E86008701403FF400413FF5000D
:10043800790886008701403FF600413FF7007708BA
:10044800803AF8007508803A7802031D2D2A74084E
:1004580076020318302A312AAA2A790886008701E9
:100468000430810741310318810A79088600870121
:10047800403FF400413FF5007908043E86008701BB
:10048800403FF600413FF7007708803AF8007508CA
:10049800803A7802031D522A740876020318552AF6
:1004A800562AAA2A7908063E860087017908083E56
:1004B80084008501403F803F413F813FAA2A790857
:1004C80086008701403FF400413FF5007508803AF7
:1004D800F60080307602031D732A01307402031C73
:1004E800762A772AAA2A790886008701FC308107AC
:1004F8004131FF30813D7F317908063E8600870112
:10050800403FF400413FF500790886008701403FED
:10051800F600413FF7007708803AF8007508803AFE
:100528007802031D992A7408760203189C2A9D2ACA
:10053800AA2A7908043E860087017908083E8400C3
:100548008501403F803F413F813FAA2A0800740847
:1005580075040319B02AB12AC22A0230F6007608B7
:100568002000A10021000D1324000D1322000D13FB
:100578000230F60076082000A000F12A20002108A9
:100588000319C72AC82ADB2A0230F6007608A00019
:100598000130A1020319D12AD22AD32AF12AA101B2
:1005A80022000D1721000D1724000D17F12A003025
:1005B8000D1B0130F7007708031DE32AE42AEC2A13
:1005C8002003031DE82AE92AEC2A8731EF27823124
:1005D8007708F60076082000A00008001230F20024
:1005E8007A30F30020004608F5004508F40084310D
:1005F8005F24823173082000B9007208B800B7017F
:100608003908803AF8008C307802031D0D2B3630FB
:100618003802031C102B112B302B20003908803A8C
:10062800F800BD307802031D1B2B09303802031C6B
:100638001E2B1F2B2D2B20003908803AF800C930BB
:100648007802031D292B3F303802031C2C2B2D2B3D
:10065800302B2000B701B70A20003708F8007808C7
:10066800A4000800F900863105268331770878044C
:1006780003193F2B402B6A2B790885316B25833171
:1006880072087304031D492B4A2B6A2B2000BE01F4
:10069800BF01772B2000491E522B542B0130552BBC
:1006A8000030C000C1014008BE004108BF00772BE0
:1006B8002000471F602B622B0130632B0030C000E5
:1006C800C1014008BE004108BF00772B7B08003AF3
:1006D80003196F2B4A2B7A08013A03194E2B033A58
:1006E80003195C2B4A2B08002D308731BF27833133
:1006F800720873040319812B822BA72B28308731AA
:10070800BF2783317208730403198B2B8C2BA72BFB
:10071800A030F2000F30F300CA30873197278331B9
:10072800A72B7030F2001730F3002D308731972750
:100738008331B42B7030F2001730F3002830873142
:1007480097278331B42B7B08003A0319AC2BB42BC1
:100758007A08013A0319952B033A03199E2BB42BF7
:100768000800F9007908860087010108031DBD2BE0
:10077800BE2BC12BF201F301F02B790A8600870109
:10078800403FF400413FF5007908033E86008701A9
:100798007208810741317308813D7F31403FF6007F
:1007A800413FF7007708803AF8007508803A7802E8
:1007B800031DE02B740876020318E32BE42BE52BCA
:1007C800BE2B7908033E860087010030C03FC13F39
:1007D8000130F2000030F3000800210095131908D9
:1007E80087396838990099131908FC390238990033
:1007F80038308C00383024008C00C03021008D0047
:10080800C03024008D00783021008E007030240024
:100818008E0023008C018D018E0121009D01260090
:100828008C018D018E018B170B178B160B11210074
:100838009512151295111508F839033895008B177C
:10084800111020001110C53098000800512C0430F8
:10085800F2000030F30032308331B523843172085E
:1008680073040319382C392C5E2C32308F31F3275E
:1008780084315E2C0430F2000030F300CF30833135
:10088800B52384317208730403194B2C4C2C5E2C4D
:10089800CF308F31F32784315E2C7B08003A03195F
:1008A800562C5E2C7A08013A03192B2C033A0319AB
:1008B8003E2C5E2C0800720873040319642C652C06
:1008C8008E2CF701F70A712C0130F235F30D890BE4
:1008D800692C0130F6007608F707F31F742C752C85
:1008E800682C73087502031D7B2C72087402031CA4
:1008F8007E2C7F2C832C7208F4027308F53B0130A0
:10090800F336F20C890B842C0130F702031D8D2C71
:100918008E2C752C7508F3007408F200080004305A
:10092800F2000030F3002D308331B5238431720892
:1009380073040319A02CA12CA52C2D308F31F3277B
:1009480084310430F2000030F30028308331B523BD
:100958008431720873040319B22CB32CB72C2830D5
:100968008F31F32784310430F2000030F300CA30AD
:100978008331B52384310800F200720886008701AC
:100988000030C03FC13F7208023E860087011E301A
:10099800C03F0030C13F7208043E86008701143012
:1009A800C03F0030C13F7208063E860087010A300A
:1009B800C03F0030C13F7208043E860087017208BC
:1009C800083E84008501403F803F413F813F080049
:1009D800F2007208860087010030C03FC13F7208EC
:1009E800023E860087010A30C03F0030C13F7208CE
:1009F800043E860087010730C03F0030C13F7208BF
:100A0800063E860087010430C03F0030C13F7208AF
:100A1800043E860087017208083E84008501403F35
:100A2800803F413F813F080020001708F400F5018E
:100A38007408B9007508BA001608F400F5017408BE
:100A4800B7007508B8001708F400F5013A087506EC
:100A5800031D302D39087406031D332D342D182D30
:100A68003A08F5003908F4007408F500F40137086D
:100A78007404F20038087504F3000800F4007408E0
:100A880086008701403F2000B700413FB800740846
:100A9800083E86008701403FB900413FBA003A0846
:100AA800803ABB003808803A3B02031D5D2D3708A9
:100AB8003902031C602D622D0130632D00302000A7
:100AC800BC00BD013C08F2003D08F3000800F4003A
:100AD800740886008701403F2000B700413FB800F6
:100AE8007408083E86008701403FB900413FBA00BC
:100AF8003A08803ABB003808803A3B02031D862D2D
:100B080037083902031C892D8B2D01308C2D0030BC
:100B18002000BC00BD013C08F2003D08F3000800BD
:100B2800F300AE2D730C2200031C8C1003188C14D8
:100B38007308F20072082000A700BB2D730C220076
:100B4800031C0E1003180E147308F200720820001C
:100B5800A600BB2D7B08003A0319B32DBB2D7A08DC
:100B6800013A0319962D033A0319A22DBB2D08004B
:100B78001230F2007A30F30020004608F5004508EC
:100B8800F40084315F24853173082000B8007208AE
:100B9800B7003808803AF800BD307802031DD62D1A
:100BA8000A303702031CD92DDB2D0130DC2D003033
:100BB800F90079082000A30008002000BA00C91E27
:100BC800E62DE82D0130E92D0030B800B9013808CC
:100BD800F2003908F3003A0882310D2285312000ED
:100BE800C81FF72DF92D0130FA2D0030B800B901D2
:100BF8003808F2003908F300370882310D228531B0
:100C080008001B2E2D308F31E72786317308F80036
:100C18007208F700282E28308F31E72786317308AD
:100C2800F8007208F700282EF701F801282E7B0833
:100C3800003A0319202E182E7A08013A0319062EB5
:100C4800033A03190F2E182E08003F2E32308F3129
:100C5800E72786317308F8007208F7004C2ECF306A
:100C68008F31E72786317308F8007208F7004C2E99
:100C7800F701F8014C2E7B08003A0319442E3C2E4C
:100C88007A08013A03192A2E033A0319332E3C2E07
:100C98000800632E20002708F400F5017408F2000C
:100CA8007508F300702E20002608F400F50174087A
:100CB800F2007508F300702EF201F301702E7B0824
:100CC800003A0319682E602E7A08013A03194E2E4D
:100CD800033A0319572E602E08002000BA00C71ED9
:100CE800762E782E0130792E0030B800B9013808F8
:100CF800F2003908F3003A0882310D2286312000CB
:100D0800471E872E892E01308A2E0030B800B9017F
:100D18003808F2003908F300370882310D2286318D
:100D280008001230F2007A30F30020004608F5007F
:100D38004508F40084315F24863173082000B80028
:100D48007208B7003808803AF800BD307802031DF1
:100D5800AF2E0A303702031CB22EB52E22008E1792
:100D6800B72E22008E130800CB2E3230F20000304E
:100D7800F3003230873197278631D82E3230F2008F
:100D88000030F300CF30873197278631D82E7B0883
:100D9800003A0319D02ED82E7A08013A0319B92E31
:100DA800033A0319C22ED82E0800F601F701721C67
:100DB800DE2EDF2EE32E7408F6077508F73D0130A6
:100DC800F435F50D890BE42E0130F336F20C890B5E
:100DD800E92E72087304031DF22EF32EDB2E77081A
:100DE800F3007608F2000800F200082F720C2200C7
:100DF800031C0E1103180E15152F720C2200031C6C
:100E08000D1203180D16152F7B08003A03190D2F24
:100E1800152F7A08013A0319FA2E033A0319012FFC
:100E2800152F0800F200262F720C2200031C0C104C
:100E380003180C14332F720C2200031C8D12031894
:100E48008D16332F7B08003A03192B2F332F7A087E
:100E5800013A0319182F033A03191F2F332F0800DB
:100E6800CA308F31DD2787317308803A2000B700F8
:100E780083303702031D422FE8307202031C452FCE
:100E8800472F0130482F00302000B800B90138083A
:100E9800F6003908F70008005B2F2D308F31F32753
:100EA8008731682F28308F31F3278731682F7B08E7
:100EB800003A0319602F682F7A08013A0319512F55
:100EC800033A0319562F682F0800742F32308F31D8
:100ED800F3278731812FCF308F31F3278731812F47
:100EE8007B08003A0319792F812F7A08013A0319F0
:100EF8006A2F033A03196F2F812F08002D308F3185
:100F0800E727873172082000B7007308B800283037
:100F18008F31E7278731720820003704F7007308FC
:100F28003804F8000800F400740A86008701720883
:100F3800C03F7308C13F7408033E86008701003034
:100F4800C03FC13F7408860087018101810A0800FB
:100F5800F200720A860087010030C03FC13F720864
:100F6800033E860087010030C03FC13F72088600FB
:100F7800870181010800F6007608860087010108CC
:100F88000319C72FC92F0130CA2F0030F400F5010B
:100F98007408F2007508F300080087313427873198
:100FA80076087704031DD92FDB2F0130DC2F0030A2
:100FB800F90079082000A500080020000C08F200BC
:100FC8007208C9000D08F2007208C8000E08F20085
:100FD8007208C70008000030F200F3008F31D527EF
:100FE80087312000C501C6010130CA000030CB009E
:060FF80008000134003482
:101F9E00640080010131890BD02F0034200018100D
:101FAE00730897007208960018140800F50075085B
:101FBE00033E86008701403FF200413FF3000800D8
:101FCE00F6007608860087010108F400F501740812
:101FDE00F2007508F3000800F2007208860087010F
:101FEE0081017208033E860087010030C03FC13F69
:061FFE0008000434003469
:020000040001F9
:04000E00E4C9FFFE44
:00000001FF
